:10014000021D800A0A5052494E540D0A80140A506A
:1001500052494E540D0A801E205052494E542022BE
:10016000544154544C4554414C45204D4F44454C0A
:100170002023223B0D208028105052494E54204D00
:100180004F44454C0D1080320A5052494E540D0ACE
:10019000803C225052494E5420222020532F4E2082
:1001A000222C20534E25313030303030303030303A
:1001B0000D2280462A5052494E542022284329209D
:1001C00031393838204F4E53455420434F4D505508
:1001D00054455220434F52502E220D2A80500A502F
:1001E00052494E540D0A805A2F5052494E542022E3
:1001F0005454424153494320222C564552532F31E7
:1002000030302C222E222C2330322C5645525325AE
:0D0210003130300D2F8064084E45570D0829
:10C000008E00FFBDF5E38621BDF8EBBDC0C842C080
:10C010002743C03044C03946C07B4DC12B50C29F1E
:10C0200052C27653C0AA00BDF8EB717F147EF9416D
:10C03000BDF8EBBDF5E37EC716BDC0E33CBDFB1408
:10C04000BDF910383CC610A600BDFB19BDF9140897
:10C050005A26F4BDF91038C610A60081202C02869D
:10C060002E817F2F02862EBDF8EB085A26EBBDF5F8
:10C07000E3BDC128812E26C47EC000BDF8EBBDF90A
:10C0800014BDC0F6183C862CBDF8EBBDC0F6DD56DD
:10C09000862CBDF8EBBDC0F637BDF5E33238A700FE
:10C0A000089C5626F9A7007EC000BDC0E3BDFB1466
:10C0B000BDF910A6009753BDFB19BDF910BDC0F620
:10C0C000E700BDF5E30820E5383CBDC128A1002705
:10C0D000096D0027F308080820F3333336EC011804
:10C0E000326E00BDF8EBBDF9147F00527F0053BDE6
:10C0F000C0F6187EF5E3BDC128812E26037EC00060
:10C10000810D2603DC5239803025EB810A25088019
:10C110000725E3811024DF9746BDFB21DC5205058E
:10C120000505DB46DD5220CE7EF8AEBDF8EBBDF551
:10C13000E3BDF87926FB71F8175FF740005CC10397
:10C1400027057C001720F371F8175FF140002738AE
:10C15000B64000363771F817CEC1754FBDF4643262
:10C160008A30BDF8EBCEC17D4FBDF464328A30BD5C
:10C17000F8EB7EC0003A2042414E4B200020524551
:10C1800041445320415320005CC10327057C001724
:10C1900020B971F817CE4002EF001805847F8B405C
:10C1A000188C400026F2CE4002AC002743DF46EE5A
:10C1B00000DF4871F817BDF5E3CEC1E14FBDF4646F
:10C1C0009648BDFB199649BDFB19CEC1E64FBDF49B
:10C1D000649646BDFB199647BDFB1971F8177EC0E2
:10C1E0000053454520002041542041444452200042
:10C1F0001805847F8B40188C400026AD8601974639
:10C2000071F81796179A469717CE40004F5FED00CA
:10C21000EC00261E4353ED00A300261F08088CC027
:10C220000026EB7C00469646810326D771F8177EE0
:10C23000C000CC0000ED00EC002007CCFFFFED00BB
:10C24000EC003C373671F817BDF5E3CEC26B4FBD3D
:10C25000F464323318BDFB148640BDF8EB383CBDA6
:10C26000FB1438EC004353ED0020F84249542045BC
:10C2700052524F522000BDF8EBBDF5E34F36323637
:10C28000BDF663DE56BDFB14BDF910324C3681405D
:10C290002709840726E8BDF5E320E3327EC000BD10
:10C2A000F8EBBDF5E37F0053BDC0F6C43F37BDF9E1
:0DC2B00010BDC0F6DD5632BDF6B37EC000F5
:10C4000000000030313030303030303030300D54BA
:10C410004154544C4554414C45204D4F44454C20CB
:10C420003320202843292031393838204F4E5345B6
:10C430005420434F4D505554455220434F52502E97
:10C440000D4C495354CB25545952554ECAC35052E2
:10C45000452A52554ECABC462452454D494E44CFFA
:10C46000A1465245D741414F4E454F4ED7E9414134
:10C4700041454F4646D7E442424E455854C941547F
:10C480004F4C4554CE885641524946CDCC4E4F5420
:10C4900045474F544FCB0D454E474F535542CD77EF
:10C4A0005352455455524ECDA0464F52C8B94745F8
:10C4B000544255525354CE985853544F5245CEDBA4
:10C4C0004150534554D3A2564150434C52D40C547E
:10C4D0004553444FDACB31313143414C4CDBF632DA
:10C4E00032434F554E54DD2845534C454550D324D7
:10C4F000525550524F47DB8E5855474554D4F94456
:10C5000046544F4E45D75C52535553454E44D47014
:10C510002F4F4E455252D6452341534DDE984A4E39
:10C520004B52454DCDBD41524B5052494E54CC56C5
:10C5300053584D4954D811574F53544F50CAB654BD
:10C540004F4954455854D6654F4F54455854D6F921
:10C55000475354494D45D82E405254494D45D891E2
:10C560004051554954D8E55245485942D968414C43
:10C570004C5653544F5245DC7956474554DCB3333F
:10C5800033494E505554CDF138585348414B45D757
:10C59000F44F46464C44D166454F4E4C4F4144DD26
:10C5A0006644494DDCE55245414E4557CAA24F4CC1
:10C5B00044434F4EDD07444545CE82544FC8DC46C8
:10C5C000524F4DF2C653544550C8F14154C8F74339
:10C5D00048414EE55A5459474554E59626474F5031
:10C5E000494EE614544845534449E98620202050DA
:10C5F0004552494F44EA6D414253E5454245455352
:10C600005152E69547415454454D50E74A484953E5
:10C61000494EE80B4F46464153494EE8774E554345
:10C620004F554E54E9D9454C4F47EB2A494E4745A3
:10C630005850ECE5495245424154E72F544F50566B
:10C64000455253E96B5A59534EE97750495A454D73
:10C650004F44454CE96253E5113DE397252F2F2ABE
:10C66000343E3DE3682F233C2F3E3CE3737E2F2A6C
:10C670003C3C3EE3732B3D2D3E3EE385454E442E30
:10C680002E3C3DE38E3F2F3E3E3CE39E3C3E3C3EF7
:10C690003CE3A58EBFFF7F00760E86FF9791BDF825
:10C6A0004C861A97111A1ABDF84C4FCE738C6F0036
:10C6B000088C73A226F87F00B37F00B4CC0C00FD79
:10C6C00072887F00B57F006A7F0076860AB7B59AC8
:10C6D000CC1770DDAF8639979F9797979497A5975A
:10C6E000A897A2867E97ABCCF8EBDDACCE73D2DFF9
:10C6F000B1FF73A2CC0000DD9ADD9C7F0077BDF511
:10C70000E386FF978C979E7F00927F00B67F009311
:10C710007EC8444F4B0D8EBFFF86FF979E860AB79B
:10C72000B59A7F00817F008CBDF5E3CEC7134FBD66
:10C73000F464CEC739FF738CCE0000FF7394FF738F
:10C740008E863EBDF8EB4FCEB294BDF374083CCE5E
:10C75000B294865CBDEDEB261EBDE2E3FC7218933D
:10C76000522607FC721A935427033820D4865CBDE6
:10C77000EDEB27037EF2C61838DF5618BDEE70DCED
:10C7800056DD4EBDEDFBDC522634DC54261B8627DD
:10C79000BDEDEB27AC7EC86B45444954494E47205C
:10C7A00044495341424C45440D7D0092270DCEC76C
:10C7B000984FBDF464BDF5E37EC7414D2A06CC0019
:10C7C000087EEF0F0909098A80ED00DF46DC4E93F1
:10C7D00046E702DE4E09E700BDF3E12705FF73AE31
:10C7E000201BFF73A6FF73AEFC73A2FD73A8BDF4FC
:10C7F00005FF73A4BDF555FC73A6FD73A2DC4E9333
:10C8000046C10526037EC741FE73A2FF73AAF373D8
:10C81000AAFD73AC188CB28F1823037EF36BFD73E3
:10C82000A2BDF56EFC73AEFD73A6DC4EFD73A8DCF5
:10C8300046FD73A4BDF5557EC741CE01006F0009CA
:10C8400026F82032B6C42E815326EFCE0142FF7364
:10C85000A4CE73D2FF73A6FC0140FD73A8BDF555AD
:10C86000FC73A6FD73A27ECABF0000CCC869FD732D
:10C870008CCCC441DD520908A600B1C42B27F8DFD7
:10C8800046A6003CDE52E6002B2811270B18C300F9
:10C890000818DF5220F0DE4A08E600DF4A38083C7C
:10C8A000E10027F2C180240838DE463CDE5220DD5C
:10C8B000DE4A08A60038363739BDF5AEBDF27EDC5B
:10C8C00052FD7394B6C42C814F2709FC73948300E6
:10C8D00004FD7394CCC5BBDD527EC876BDE2E3DCBB
:10C8E00054FD7398DC52FD7396CCC5C5DD527EC8ED
:10C8F00076BDE2E37EC900CC0001DD545F4FDD521E
:10C90000DC52FD739ADC54FD739CFC738CFD739EAA
:10C91000FF73A030200518C3000E18EC00271C1868
:10C92000BC73941826F0FF73AA18C3000EFD73ACF5
:10C9300030FF73AEBDF56EFE73AC35FE73A07EEEB8
:10C9400002BDEE0824037EF2C6FD73903CFE739494
:10C950002604387EF2C6BC7390270738BDF5877E63
:10C96000C94CEC02F3739CED02EC00F9739BB973B4
:10C970009A295BED00FC739A2B267D73962A066D2F
:10C98000002A4D20046D002B39EC0018BC7396254D
:10C9900031263D18EC0218BC739825262724203038
:10C9A0007D73962B066D002B2720046D002A13EC57
:10C9B0000018BC73962519260918EC0218BC739848
:10C9C000250E38FC739EFD738CFE73A02006ED00CF
:10C9D00038BDF5877EEE02BDE2E3DC522605DC546D
:10C9E0004D2A09CC00087EEF0F7EF2C63637862C22
:10C9F000BDEDEB26F4BDE2E3DC5226E7DC544D2B23
:10CA0000E23332DD48DC54934825D83CFE738CEC8D
:10CA100000847FDD502733189C48252E9C54270224
:10CA20002428BDF5E3CECA304FBDF464387EC71666
:10CA300043414E4E4F542045524153452043555299
:10CA400052454E54204C494E450DDE54DF52DE48CF
:10CA5000DF54CE73D2BDF3F32404387EEE02FF73AD
:10CA6000A6DC52C30001DD54BDF3F32408FC73A619
:10CA7000FD73A22012FF73A4FE73A2FF73A8BDF57D
:10CA800055FE73A6FF73A2DE5027CFDF54CE73D2BC
:10CA9000BDF3F3080808A600810D27BF813A27BB24
:10CAA00020F3BDEDFB810D2707813A27037EC9D70F
:10CAB000CC73D2FD73A2BDF2BB7EC716BDF2BB869E
:10CAC000FF2004BDF2BB4F978C7F0081CE73D27FD5
:10CAD00000547F0055BDF3F324037EC716FF738C0B
:10CAE00096B5271BBDF8EBEC00847FDD547F005228
:10CAF0007F005386019745BDF49F863EBDF8EB0845
:10CB00000808BDF5F4CCC479DD527EC876BDE2E3F9
:10CB10003CBDF2BBBDF418270738CC00157EEF0FE3
:10CB200032327ECADDBDEE0824037ECBC23CFD73EB
:10CB3000AA18EC00DD64EC02DD66CCEFD9DDAC3880
:10CB40007F00547F0055862CBDEDEB260DBDEE70A9
:10CB5000DC522706CC00087EEF0FDC542BF636376C
:10CB600096442729862CBDEDEB270A862DB1C42ECD
:10CB7000BDEDEB2613BDEE7096442711DC5226D492
:10CB8000DC542BD0DD5E200ACC00002003CC7FFFDC
:10CB9000DD5E3332DD543CBDF3E12512BDF530BD21
:10CBA000F3F3250AEC00847F935E27F025EEFE73F5
:10CBB000AADC64ED00DC66ED02CCF8EBDDAC387E7F
:10CBC000C716BDEE70DC522706CC00087EEF0FDCE6
:10CBD000542BF6363796442729862CBDEDEB270AD1
:10CBE000862DB1C42EBDEDEB2613BDEE7096442705
:10CBF00011DC5226D4DC542BD0DD5E200ACC0000A0
:10CC00002003CC7FFFDD5E3332DD5496763686011D
:10CC100097763CBDF3E12517BDF5307D0093262ABC
:10CC2000BDF3F3250AEC00847F935E27EB25E938FA
:10CC30003284019776863BBDEDEB260BBDF8AE81C5
:10CC40001327F9811127F57EC716383284019776AC
:10CC5000BDF84C7EC716863BBDEDEB26037EEE028B
:10CC6000860DBDEDEB270C863ABDEDEB27058D0A51
:10CC70007EEE0209BDF5E37EEE0286019745BDF426
:10CC80007827698623BDEDEB2639C600A6008130E2
:10CC90002602C680D745BDE2E39655847F9A459724
:10CCA000458648C610A10027138642C602A1002768
:10CCB0000B8651C608A1002703C60A0908F7B59AD2
:10CCC0007ECCECA600815C260A08BDE2E396559D69
:10CCD000AB2019867BBDEDEB260CBDCD11867DBD4D
:10CCE000EDEB26252006BDE2E3BDF49F862CBDEDCD
:10CCF000EB278B863BBDEDEB260139860DBDEDEBB9
:10CD0000270A863ABDEDEB27037EF2C6BDF5E3099F
:10CD100039BDE2E3BDCF7ADC523637DC5436378694
:10CD20002CBDEDEB26E3BDE2E3BDCF7A3332DD4827
:10CD30003332DD469352250E2706CC00167EEF0FC8
:10CD4000DC54934825F4BDCD60BDF044BDCD609D5D
:10CD5000ABDC46935225EF2606DC54934824E73992
:10CD60003CDE463CDE483CDE64DF46DE66DF4838BB
:10CD7000DF6638DF643839BDF5AEBDE2E3BDF2BB36
:10CD80003CBDF418270738CC00157EEF0F18FE7352
:10CD90008C3CFE738E3C7F7394BF738E187ECADD0D
:10CDA000BDF2BBFC738E26037EF2C6BE738E38FFC7
:10CDB000738E38FF738C38BDF5877EEE02FE738C60
:10CDC0007F00547F0055BDF4057ECAD8BDE2E3DC88
:10CDD000522604DC5427037ECB02BDF40F25037ECC
:10CDE000CADD7EC716BE739238FF738C3838BDF526
:10CDF000E33CBDF4782609BDEE08DD542568202308
:10CE00003CBDEE08DD5424037EF2C6A600B1C42D5D
:10CE100097454FA70038BDF464964509A700863AA8
:10CE2000BDF8EB3CFE738C3CCEFFFFFF738CBF73F1
:10CE300092DC543736863ACEB394BDF374CEB394B5
:10CE4000A600810D2606A7018630A700BDE2E3BD3E
:10CE5000EDFB810D268F380FDC54ED02DC52ED0026
:10CE60000E38FF738C3832B1C43132863BBDEDEBE6
:10CE70002703BDF5E3862CBDEDEB26037ECDF17EC9
:10CE8000EE02A600810D270ABDF27E862CBDEDEBD9
:10CE900027F67EEE027EF2C6BDCF61862CBDEDEB9D
:10CEA00026F3BDE2E33CDE522609DE5427058C0062
:10CEB00009250738CC000B7EEF0F18D7467F0047B7
:10CEC000D6474FC3E58E18E600BDF71617BDEFD95C
:10CED0007C00479647914626E7202CBDCF618631DE
:10CEE0009762862CBDEDEB261D8623BDEDEB26312A
:10CEF000A600088132270B81342707813127037E62
:10CF0000F2C6976220DC3CFE73AAB6C42D814E2780
:10CF100004DC422002DC66ED02DC64ED00387EEECB
:10CF200002BDEDFB8127270481222610CCEFD9DD3D
:10CF3000ACBDCC7ACCF8EBDDAC7ECF06BDE2E3D65F
:10CF400062C134260C9652BDEFD99653BDEFD9205D
:10CF500004C13226059654BDEFD99655BDEFD920B0
:10CF600081BDEE082511FD73AA3CFE73AAEC00DD1D
:10CF700064EC02DD6638397EF2C6CC0001DD46CCB9
:10CF80000000D39CDD48DC46D99B999A9352250B2F
:10CF90002608DC4893542503270139CC00167EEF80
:10CFA0000F3CFC73A28373D22604387EEE02188CE9
:10CFB0003EBF2534CECFBE4FBDF4647EC71650525F
:10CFC0004F4752414D20544F4F2042494720464F32
:10CFD0005220524F4D202831363338322042595496
:10CFE0004553204D4158290018C30142FD73D0CE4E
:10CFF000D2F74FBDF464BDF5E3CE17701ABDF874D7
:10D00000260D0926F7CED3074FBDF4647EC716BDA3
:10D01000F8AE811826037EC7168115268DCEB5FF82
:10D02000DF5286019755FC73A2DD4ACC8D70DD4C32
:10D03000CE73D0BDD07038862BBDEDEB3C260C4FA7
:10D040005FDD4CDD4ACEC000BDD0704FCED05BA6B8
:10D050000081242714BDD0F20820F43A303030305B
:10D060003030303030300D0A24BDD143387EEE02EE
:10D07000DF4E7F00467C0046089C4A270696468184
:10D080001026F2863ABDD0F27F00479646BDD0D139
:10D09000DC4ED34C37BDD0D132BDD0D14FBDD0D175
:10D0A000DE4EA600BDD0D1089C4A27107A00462645
:10D0B000F14F9047BDD0D1BDD0C620B44F9047BDF1
:10D0C000D0D1BDD0C639860DBDD0F2860ABDD0F212
:10D0D00039369B47DD47323644444444BDD0E432C0
:10D0E000BDD0E439840F8B30813A25028B07BDD047
:10D0F000F2393CDE52A7008CB67E270608DF523894
:10D10000393CCEB5FFDF524F97548601BDF8EB9600
:10D1100055BDF8EB43BDF8EBA600BDF8EB9B54976B
:10D1200054088CB67F26F19654BDF8EBBDF8AE815D
:10D130001527CF810626CB811826037EC7167C00D3
:10D14000553839DE528CB67F270B6F00088CB67FBE
:10D1500026F8BDD1018604BDF8EBBDF8AE811827D5
:10D16000DA810626DE39BDE2E3BDCF7ADC52DD642A
:10D17000DC54DD66862CBDEDEB27037EF2C6BDE2F6
:10D18000E3BDCF7ABDD2EC2406CC00167EEF0FB6FD
:10D19000C42E81532708DC529A40DA41DD5218DE52
:10D1A000523CDE543C18862CBDEDEB2707CC1770A3
:10D1B00036372020BDE2E3DC522706CC00177EEF95
:10D1C0000FDC543637862CBDEDEB2608BDEE082467
:10D1D000067EF2C6CC004EDD4E3332DD501838DF0D
:10D1E0005438DF52183CDE4E8C004E260ACED2F761
:10D1F0004FBDF464BDF5E3BDD2102620DE4E8C0099
:10D200004E260ACED3074FBDF464BDF5E37ED2DED1
:10D21000DE501ABDF87426030926F739BDF8AE8131
:10D220001826037ED2DE811526CD8601974720344D
:10D230007C0047BDD210260D3338BDD2EC24037ECE
:10D24000D2BE7ED2DEBDF8AE3338810627168118F5
:10D2500026037ED2DE811527043C3720D6DF66D731
:10D26000657A0047BDD2EC254BDE663CD665377F3C
:10D27000005A7F005B8601BDF8EB9647BDF8EB4393
:10D28000BDF8EBBDD2EC2515965A8180271EBDF066
:10D2900044BDF8EB9B5B975B7C005A20E6965A8175
:10D2A0008027094FBDF8EB7C005A20F1965BBDF852
:10D2B000EB7ED2308604BDF8EBBDD2102619730088
:10D2C00064730065DC664353C30001DD66DC64C93A
:10D2D000008900DD642007BDF8AE810626D6DE4E4B
:10D2E000DC64ED00DC66ED02387EEE02965390655C
:10D2F0002604DC5493663957414954494E47204629
:10D300004F52204E414B004E414B204E4F54204631
:10D310004F554E44204245464F52452054494D45B5
:10D320004F555400BDE2E3DC522706CC00187EEFD7
:10D330000FDC54260D96431A914327FB4FDD6C7E7C
:10D34000EE02DD6E200108A600B1C43127F8813A53
:10D35000272C810D27283C20091ADC6C936E270BA3
:10D3600024097B401527F2387ECB02DD6C38CC00D7
:10D3700000DD54BDF40F25037ECADD7EC7163C1ABE
:10D38000DC6E936C270925022AF5862ABDF8EBCEC0
:10D390000000DF6C387EEE029DA53838CC000C7E94
:10D3A000EF0FBDE2E3DC52270DCC000C7EEF0F3C0B
:10D3B0008DE6387EEE02DC544D26F4C10E24F0C119
:10D3C00008241786805D2704445A20F9369A159759
:10D3D00015329A8B9720978B201EC00886805D2778
:10D3E00004445A20F9B1C43124024444369A0397C4
:10D3F00003329A8A9701978A862CBDEDEB27A37E8C
:10D40000EE029DA83838CC000C7EEF0FBDE2E3DCC5
:10D4100052270DCC000C7EEF0F3C8DE6387EEE02DD
:10D42000DC544D26F4C10E24F0C108241886805D1A
:10D430002704445A20F9364394159715329A8B974E
:10D4400020978B2021C00886805D2704445A20F94C
:10D45000B1C43124024444364394039703329A8A78
:10D460009701978AC00E862CBDEDEB279F7EEE02BA
:10D47000BDD5DF86809A8A9701978ABDEDFB812210
:10D48000270481272610CCD4CCDDACBDCC7ACCF8D7
:10D49000EBDDAC7EEE02BDD61FDC7B2604DC7927FB
:10D4A0001BBDF044BDD4CCDC7B830001DD7BDC798B
:10D4B000C2008200DD7926E9DC7B26E53CFE73AA0A
:10D4C000DC64ED00DC66ED02387EEE023CDE7D8C35
:10D4D000011324010FBDD5D9717F03BDD5D9C6086D
:10D4E000442505717F0320057280032000BDD5D936
:10D4F0005A26ED728003380E39BDD5DFBDD61F86A2
:10D500002CBDEDEB27037EF2C6BDE2E3DC7B2607F4
:10D51000DC7926037ED4BC86FE948B9720978B867D
:10D520007EB7010CCCD58AFD010DDC522706CC005C
:10D53000257EEF0F0FDC42D354DD54DC40D95399E4
:10D5400052DD5296AE8900974E7F007FDF467F0006
:10D5500080DC7D83011325037A00800E01010F72A8
:10D5600001140E1A0F967F2616964E90AE251026A1
:10D57000EADC529340250826E2DC54934224DC7115
:10D58000FE140E86FF97807ED4BC71FE1496802711
:10D59000010EDC7D04D37D18BDD5DBC68096150455
:10D5A00025070101BDD5D920F417DE46BDEFD9DC32
:10D5B0007B830001DD7BDC79C2008200DD79DC7DCC
:10D5C00004047B0115260583000126F6DC79260874
:10D5D000DC7B260486FF977F3BDE7D0926FD39BD77
:10D5E000E2E33CDC52DD46DC54DD48BDEF8ECC048A
:10D5F000B0DD53BDF086DC52260CDE548C0FA02427
:10D60000058C001E240A38CC00197EEF0F7EF2C66E
:10D6100018830007DD7D38862CBDEDEB26EF39BD84
:10D62000E2E3DC52DD79DC54DD7B862CBDEDEB26BC
:10D63000DCBDEE0825D7FD73AA3C18EC00DD64ECD8
:10D6400002DD663839BDE2E3BDF2BB3CBDF418270C
:10D650000A387F0081CC00157EEF0FDF823886FF0D
:10D6600097817EEE02BDCF61860DB773AC862CBD6F
:10D67000EDEB2616865CBDEDEB2636BDE2E3965556
:10D68000B773AC862CBDEDEB27273C4FCEB394F699
:10D6900073ACBDF376CEB394A600B173AC270C087F
:10D6A000DF5238BDEFD93CDE5220EDBDEFD97ECF41
:10D6B00007BDE2E3DC522706CC001A7EEF0FDC54F4
:10D6C000272ADC54DD52BDF874270FBDF8AE36BDF5
:10D6D000EFD932B173AC271120EC1ABDF87426E2F1
:10D6E000DC52830001DD5226F17ECF06BDF874279F
:10D6F000F8BDF8AEBDEFD920F0BDCF61860DB77390
:10D70000AC862CBDEDEB2612865CBDEDEB27037ECF
:10D71000F2C6BDE2E39655B773AC3CBDF044B173BD
:10D72000AC2705BDF5E520F33836863BBDEDEB3281
:10D73000270C810D2605BDF5E32003BDF8EB7ECF58
:10D7400006BDF2BBCCB28FB373A2DD547F00527F13
:10D75000005386069745BDF49F7EC716BDE2E3DC05
:10D76000522706CC001B7EEF0FDC54188C006E187D
:10D7700025F13637862CBDEDEB26E8BDE2E3DC5221
:10D7800026E1DC5426043232203A05DD5425D43318
:10D7900032DD463C867EB70106CCD7C7FD01077156
:10D7A000FD03CC0000DD09DE46DF0B9608DF0B86AB
:10D7B00001970F860897081ADC4626FB7F0008862B
:10D7C00000970F387EEE029608DE54270E09DF54CC
:10D7D00088019708DC0BD346DD0B3BDC0BD346DD21
:10D7E0000BDF463B86FF3620024F36BDF2BB329739
:10D7F000927EC716BDE2E3DC522706CC001C7EEF0A
:10D800000FDC542706DDAF860120014F97767EEEB0
:10D8100002A600812D260DBDF87926FB86FF08970C
:10D82000777EEE02812B27037EF2C64F20F07F0029
:10D8300017722017720817C6A0BDF788F673B3D702
:10D840008D8D2CF673B7D78E8D25F673BBD78F8D44
:10D850001EC601BDF788F673BF8D14F673C38D0F16
:10D86000F673C78D0A71DF17868097177EEE024F19
:10D87000C00A4C24FB4ACB0A484848481B167EF78E
:10D8800088BDF7671784F044364444C40F1B331B2C
:10D89000393CCE73B06F00088C73C826F8387F000F
:10D8A00017722017720817C620BDF78886EB9716E7
:10D8B000BDD881B773B3BDD881B773B7BDD881B7B1
:10D8C00073BBBDF767BDD881B773BFBDD881B773D0
:10D8D000C3BDD881B773C786FB971671DF178680E3
:10D8E00097177EEE029617840427037EEE02BDD9B9
:10D8F000199752860A1A4A26FCBDD919964991529F
:10D9000027F1BDD9473CB6C434BDF9DF389617843A
:10D910000427F2BDF84C7EEE027F001772201772CA
:10D920000817F6C431BDF78886EB9716BDD88197E6
:10D9300049BDD8819748BDD8819747C6FBD7167196
:10D94000DF17C680D717397F0017722017720817A4
:10D95000C630BDF78886EB9716BDF76771DF17C62F
:10D9600080D71786FB971639BDE2E3DC522706CC39
:10D97000001F7EEF0FDC542709188C80001824EF5D
:10D980002012BDDAAB9649978D9648978E964797A9
:10D990008F7EEE02BDDA8ADC50D354DD54D64FC9F7
:10D9A00000D753BDDAABBDDA66DC53935F250C2696
:10D9B00011965590612504260920CA862ABDF8EBE8
:10D9C00020C3DC5F934F250A2617966190512502EC
:10D9D000200FDC60C35180DD60965F8901975F2076
:10D9E000C87B041727128655D6431AD14327F94A14
:10D9F00026F6BDF5F47ED9A3DC549360188C000A9A
:10DA0000182502C60ADB49D749C03C2518D7497CEE
:10DA100000489648803C250D97487C0047964780F3
:10DA20001825029747BDD9477F0017722017720843
:10DA300017F6C42CCB59BDF788D649BDD86FD64848
:10DA4000BDD86FD647BDD86F71DF17C680D7173CDA
:10DA5000DE523CDE543CB6C435BDF9DF38DF543805
:10DA6000DF52387ED9A6BDD9199648C63C3DDB4960
:10DA70008900DD609647C6103DD360DD609647C6DD
:10DA80000E3D7F005FD35FDD5F39968EC63C3DDB88
:10DA90008D8900DD50968FC6103DD350DD50968F96
:10DAA000C60E3D7F004FD34FDD4F39BDD919964982
:10DAB0009752860A1A4A26FCBDD9199652914927CF
:10DAC000F139CC00207EEF0F7EF2C6BDEDFB812246
:10DAD000270481272613BDDB7ACCDB5DDDACBDCC12
:10DAE0007ACCF8EBDDAC7EEE02BDE2E318DE523C10
:10DAF000DE543C18862CBDEDEB26CDBDE2E3DC52B6
:10DB000026C0965426BCD6552750C12124B4BDDB6F
:10DB10007AD7461838DF5438DF5218D64686209018
:10DB200046270F7800557900547900537900524AFE
:10DB300020EF7B80522705720403200371FB0372E0
:10DB4000041571FB1578005579005479005379005C
:10DB5000525A26DE72201571DF157EEE02C6084984
:10DB60002405720403200371FB0372041571FB1575
:10DB70005A26EC72201571DF153986049A8A9701AE
:10DB8000978A86249A8B9720978B71DB1539862785
:10DB9000BDEDEB270A8622BDEDEB27037EF2C6BD65
:10DBA000DBCA974EBDDBCA36BDDBCA1632DD46BDC9
:10DBB000DBCABDDBCAD64E270E5AD74E3CDE46A77F
:10DBC0000008DF463820EB7EEE028D0A48484848C0
:10DBD000368D03331B39A600088030250C810A25B9
:10DBE0000B80072504811025037EF2C639CC002165
:10DBF0007EEF0F7EF2C6BDE2E3DC5226F0DC541865
:10DC00003C18862CBDEDEB26EABDEDFB81222704F6
:10DC100081272610183818DDACBDCC7ACCF8EBDDA6
:10DC2000AC7EEE02BDE2E318DE523CDE543C1886C8
:10DC30002CBDEDEB2705CC004E2005BDEE0825B32D
:10DC4000FD73AA1838DF5438DF5238DF46183CBD60
:10DC5000F87926FBCEDC603CDE463CDC54DE5239F3
:10DC60003CFE73AAED02183818ED00387EEE027EF5
:10DC7000F2C638CC00247EEF0FBDEE0825F13C182B
:10DC80008C719C25EDEC00DD56EC02DD541883729E
:10DC9000184353C30001541736BDF6B3DC54DD56A8
:10DCA000324CBDF6B3387EEE027EF2C638CC00248C
:10DCB0007EEF0FBDEE0825F13C188C719C25ED3CE4
:10DCC000188372184050C30001541736BDF663DC48
:10DCD00056DD52324CBDF66338DC56ED02DC52EDB7
:10DCE00000387EEE02BDE52FDC522615DC54188C80
:10DCF0000014250C8C0C01240718FD72887EEE029E
:10DD000018CC00237EEF0F7F00B37F00B4867BBD6D
:10DD1000EDEB260EBDEE08250CDDB3867DBDEDEBEB
:10DD200026037EEE027EF2C67F0008BDEE08251CAB
:10DD3000FDB598867EB70109CCDD4FFD010AC6020C
:10DD4000D708D608DC0DDC09C612D7087EEE02968D
:10DD500008FEB598EC02C30001ED02EC00C9008991
:10DD600000ED00DE0D3B86FF974F860197503CCCBF
:10DD70000052FD73ACBDEE0825123637862CBDED82
:10DD8000EB26073332FD73AC2002323338BDE2E3B9
:10DD9000DC52DD64DC54DD66862CBDEDEB27037EB2
:10DDA000F2C6BDEE0825F8FD73AA3C96B636861875
:10DDB00097B6BDF84CCE006496431A914327F9BD3F
:10DDC000F87426EE0926F18615BDF8EB7C004FD6D7
:10DDD0004FC11426208618BDF8EBFE73AA4FED0242
:10DDE0005FED00FE73ACDC66ED02DC64ED003297A3
:10DDF000B6387EEE02BDDE7A27CDBDF8AE8118269C
:10DE000004C61520D5810426098606BDF8EBD64F39
:10DE100020C88101269CBDDE2526978606BDF8EB2D
:10DE20007C005020D0CEB394C683BDDE6AA7000824
:10DE30005A26F7FCB3945311270139CEB3964FAB52
:10DE400000088CB41626F8B1B416270139B6B3947D
:10DE50004C915026064A9150270139CEB396A60020
:10DE6000BDEFD9088CB41626F5393CBDDE7A3827CB
:10DE700004BDF8AE3938387EDDB2CE01F4BDF87499
:10DE800027013996431A914327F90926F03938CCEE
:10DE900000017EEF0F7EF2C6BDEE08240ABDEE70D3
:10DEA000964427F1CC0052FD73AA3C18EC0026DE04
:10DEB000EC02FD73AC38862CBDEDEB26D87EDED4AB
:10DEC000863BBDEDEB27F63CFE73AAFC73ACED027E
:10DED000387EEE02CCE101DD46BDEDFBDF483CDEE5
:10DEE00046A100260908DF463808A60020F0A60053
:10DEF0002B1908A6002AFB0808A6002604387EF283
:10DF0000C6DF4638DE48A6007EDEDE3C16584FC32C
:10DF1000E0EB18EC00186E0038A601BDE0DF387E9B
:10DF2000DEC038A601BDE0DF38BDE2E3DC522703E6
:10DF30007EEF0FDC542718830001B373AC4D260627
:10DF4000C18024EC200881FF26E6C18025E217BDB0
:10DF5000E0DF7EDEC038A60138E600C1412706C1F9
:10DF60004226058B100820E736BDE2E3BDE0A62778
:10DF70000C328B30BDE0DFBDE0C07EDEC032BBC402
:10DF800031BDE0DFBDE0CB7EDEC038A6013836BD56
:10DF9000E2E3DC5227037EEF0FDC544D26F8378690
:10DFA0002CBDEDEB27037EF2C6BDE2E3DC5226E694
:10DFB000DC544D26E1BDE0A62616DF46183332BDFF
:10DFC000E0DF17BDE0DF1817BDE0DFDE467EDEC014
:10DFD000DF461833328B107EDFBF38A601387EDF74
:10DFE0006838A60138E600C1412709C14227037EEF
:10DFF000F2C68B4036088623BDEDEB262EBDE2E34C
:10E0000032BDE0DFBDE0CB7EDEC038A6013836B6DB
:10E01000C42D802BBDEDEB2612BDE2E332BDE0DF67
:10E02000BDE0C07EDEC038A6013836BDE2E3BDE00B
:10E03000A6260C328B20BDE0DFBDE0CB7EDEC09695
:10E0400054270C328B30BDE0DFBDE0C07EDEC03235
:10E050008B1020E238A601BDE0DF38BDE2E3BDE071
:10E06000CB7EDEC038388622BDEDEB2604167EE07E
:10E07000798627A100260D1608A6000811270BBDDA
:10E08000E0DF20F5BDE2E3BDE0CB862CBDEDEB2764
:10E09000D57EDEC03838BDE2E3BDE0C0862CBDEDE4
:10E0A000EB27F37EDEC0A600B1C42B26030820F6C2
:10E0B000812C260B08A60008815827037EF2C6395A
:10E0C000DC52260E9654BDE0DF200EDC522706CC33
:10E0D00000277EEF0F965426F99655BDE0DF393CB8
:10E0E000FE73ACA70008FF73AC3839DF18DF22DFFE
:10E0F00055DF8ADFDADFE1E00AE026E054E064E0A1
:10E10000944E4F5080014C535244800441534C4430
:10E11000800554415080065450418007494E588034
:10E12000084445588009434C56800A534556800B95
:10E13000434C43800C534543800D434C49800E5360
:10E140004549800F53424180104342418011544160
:10E150004280165442418017584744588018444121
:10E16000418019534C50801A414241801B545358EE
:10E170008030494E53803150554C41803250554C7F
:10E18000428033444553803454585380355053486B
:10E1900041803650534842803750554C5880385251
:10E1A00054538039414258803A525449803B50532D
:10E1B0004858803C4D554C803D574149803E53570F
:10E1C00049803F425241812042524E81214248497A
:10E1D0008122424C53812342434381244243538151
:10E1E00025424E458126424551812742564381288A
:10E1F000425653812942504C812A424D49812B423B
:10E200004745812C424C54812D424754812E424C2B
:10E2100045812F4E45478240434F4D82434C5352D8
:10E220008244524F528246415352824741534C825C
:10E2300048524F4C8249444543824A494E43824C9E
:10E24000545354824D434C52824F41494D83614F48
:10E25000494D836245494D836554494D836B4A4D11
:10E2600050844E5355424486834144444486C343BC
:10E270005058868C4C444486CC4C4453868E4C4437
:10E280005886CE5355428580434D50858153424335
:10E290008582414E44858442495485854C4441855C
:10E2A00086454F52858841444385894F5241858A2E
:10E2B000414444858B53544141878753544142879D
:10E2C000C7535453878F4A5352878D53544487CD35
:10E2D00053545887CF425352888D44428900445743
:10E2E0008A0000BDE313F6C431A600081127FA81A5
:10E2F0007C27020939DC543736DC523736BDE3134C
:10E3000032339A52DA53DD5232339A54DA55DD54AD
:10E310007EE2E6BDE343F6C42BA600081127FA818E
:10E320002627020939DC543736DC523736BDE34341
:10E3300032339452D453DD5232339454D455DD5495
:10E340007EE316BDE3E9A60008B1C43A27F80981C7
:10E350003C2504813F250139DC543736DC52373601
:10E36000CCC659DD527EC876BDE3AE250B8601973B
:10E37000552008BDE3AE26F57F00557F00547F0091
:10E38000537F005239BDE3AE27EE25EC20DFBDE31D
:10E39000AE27DA25D820E1BDE3AE26DC20CFBDE3F1
:10E3A000AE24D520C83233DD523233DD5439DF4E4E
:10E3B000381838DF5038183C183CDE503CDE4EBD73
:10E3C000E3E93233DD463233DD4896469852182A67
:10E3D0000CDE529C462610DE549C481839DE469CC2
:10E3E000522604DE489C541839862DBDEDEB2606D6
:10E3F000BDEF8E7EE442862BBDEDEBBDE453862B54
:10E40000BDEDEB2635DC543736DC523736BDE453F0
:10E410003233DD463233DD48DC54D348DD54DC5240
:10E42000974ED9479946DD52964E98462BD0964E38
:10E4300098522ACACC00097EEF0F862DBDEDEB273E
:10E440000139DC543736DC523736BDE453BDEF7644
:10E450007EE410BDE4E7862ABDEDEB2621DC5236D2
:10E4600037DC543637BDE4E73332DD483332DD463E
:10E47000BDF164DC4EDD52DC50DD547EE456A60076
:10E48000812F270581252701393C087F00447D0025
:10E49000522A067C0044BDEF76DC523637DC543617
:10E4A00037964436BDE4E73297447D00522A067A17
:10E4B0000044BDEF76DC52DD46DC54DD483332DD0E
:10E4C000543332DD523CBDF08638183836A6008110
:10E4D000252608DE4EDF52DE50DF543218964427E0
:10E4E00003BDEF767EE4560908A600812027F98156
:10E4F000302504813A25308128273E81262728A609
:10E50000018141250C815B2408CCC5CFDD527EC83A
:10E5100076BDEE08DD52251E3C0FDE52EC00DD52CA
:10E52000EC020EDD543839BDEE709644270839866A
:10E5300028BDEDEB27047EF2C608BDE2E38629BDC7
:10E54000EDEB26F239BDE52F96522A03BDEF769604
:10E55000522B0139CC000A7EEF0FBDE52FDC52278C
:10E5600006CC000B7EEF0F3C8D0738DD545FDD528B
:10E5700039DE548C0008250A9D9F3838CC000B7E6C
:10E58000EF0F18C3E58E18E600BDF7164F391F1BB5
:10E590001E1A1D191C1818FE73AA3CDE643CDE66A8
:10E5A0003C188628BDEDEB2629BDCF617F00527F48
:10E5B00000537F0054862CBDEDEB26288623BDED4D
:10E5C000EB260FA600088134270B813227118131F9
:10E5D00027127EF2C6BDF0449752BDF0449753BD5A
:10E5E000F0449754BDF04497553CFE73AADC66EDA9
:10E5F00002DC64ED00381838DF6638DF6438FF73FA
:10E60000AA188629BDEDEB26C9399DA23838CC0061
:10E610000C7EEF0F8628BDEDEB2657BDEF8EDC5448
:10E62000053736BDE2E3DC52270CCC000C7EEF0F41
:10E630003C8DD7382021DC544D26F5C10E24F1C184
:10E6400008243386805D2704445A20F93643948B8E
:10E650009720978B32941527073233C3000120028D
:10E660003233DD54862CBDEDEB27B38629BDEDEBAF
:10E6700027037EF2C639C00886805D2704445A20ED
:10E68000F9B1C43A240244443643948A9701978AE4
:10E6900032940320C2BDE52F96522A06CC000D7E8F
:10E6A000EF0FCC0000DD46DD48DD4EDD50DD4CCC0B
:10E6B0004000DD4A860F975ADC48D350DD58DC46CF
:10E6C000D94F994EDD56DC58D34CDD58DC56D94B2A
:10E6D000994ADD5674004E76004F76005076005110
:10E6E000DC529356251E2606DC5493582516DC561C
:10E6F000DD46DC58DD48DC50D34CDD50DC4ED94BD8
:10E70000994ADD4E74004A76004B76004C76004DF7
:10E7100074004A76004B76004C76004D7D005A26F8
:10E7200009DC4EDD52DC50DD54397A005A20893C38
:10E73000BDEF8EC61CBDF716D7547F00467F00473D
:10E74000CC028DDD48BDF0863839BDE52FDC52277F
:10E7500006CC000E7EEF0FDC544D26F517C4FC10DE
:10E760005497464FC3E7893C18EC00DD4EA3029650
:10E77000463DCB0204044353C30001D34EDD542A6B
:10E7800006730052730053383905DC05DC055A0462
:10E79000AB043603DF038E0353032102F402CD02E0
:10E7A000A90288026A024E0233021A020301EC0136
:10E7B000D701C201AE019B018901760165015401B7
:10E7C00043013201220112010200F200E200D300F3
:10E7D000C400B400A40095008500760066005600D1
:10E7E000460035002400130001FFEEFFDCFFC8FFE8
:10E7F000B3FF9DFF86FF6DFF53FF35FF15FEF0FE53
:10E80000C4FE8FFE48FE1BFE1BFE1BBDE52F3C7D9C
:10E8100000522A09DC545343C38001DD54DC548484
:10E820007FDD52188C4000182505CC80009352DD06
:10E8300046164F05C3E8E018EC00DD48EC02A300E3
:10E84000974E96473D97517F0050D64E96473DD301
:10E8500050D3487F00527F00537D00542A15435304
:10E86000730052730053C3000118DC52C9008900C1
:10E87000DD5218DD543839BDE52F3C7F00567D0050
:10E88000522A06BDEF767A0056DC52270738CC00B4
:10E890000F7EEF0FDC5427462BF3CEE8E07F0057C6
:10E8A000EC00189C5418240708087C005720F1DD60
:10E8B0004A0909EC00DD4CDC4A934CDD48CE0000EF
:10E8C000DF46DC54934CDD537F0055BDF0869657F0
:10E8D0004A5FD354DD547D00562703BDEF763839A7
:10E8E000000003240648096A0C8C0FAB12C815E21D
:10E8F00018F91C0B1F1A2223252828262B1F2E103F
:10E9000030FB33DE36BA398C3C563F1741CE447A61
:10E91000471C49B44C3F4EBF5133539A55F55842AA
:10E920005A825CB35ED760EB62F164E866CF68A69A
:10E930006A6D6C236DC96F5E70E2725473B57504B5
:10E940007641776B788479897A7C7B5C7C297CE35F
:10E950007D897E1D7E9C7F097F617FA67FD87FF5A4
:10E960007FFFCC0003DD545FDD5239FCFFE8DD544E
:10E970007F00527F0053393CCEC403BDEE7038395E
:10E98000CC00107EEF0FBDE52FDC5226F396542607
:10E99000EFD655BDEF8E5D27E7C12124E386BF94F6
:10E9A0008A9701978A968B8A14978B972071EB151B
:10E9B00072101520127800557900547900537900AF
:10E9C0005272041571FB157B400327037C00555AD6
:10E9D00026E339CC00117EEF0FBDE52FDC5226F384
:10E9E000DC5427403C18968A84FE9701978A867EDD
:10E9F000B70109CCEA25FD010A7F00547F00559636
:10EA0000431A914327FB01010101D608DC0D96430F
:10EA1000C6120FD7080E1A914327F796430926F21C
:10EA20007F00083839960884EF9708DC0DDC54C362
:10EA30000001DD54DC52C9008900DD523B9608DE3E
:10EA40004A08DF4A84E29708DE0DDF54B4C42B275E
:10EA50000EDE548C80002407DE5208DF52DC093BB6
:10EA6000960820F47EF2C6CC00127EEF0F8628BDF9
:10EA7000EDEB26F0BDE2E3DC5226ECDC5427E8188F
:10EA80003C18862CBDEDEB26DBBDE2E3DC5226D73D
:10EA9000DC5427D3DD4E183818DD508629BDEDEB48
:10EAA00026C23C968A84FE9701978A867EB7010922
:10EAB000CCEA3DFD010A867EB70103CCEA60FD0188
:10EAC000047F004A7F004B7F004CC602D708CC0071
:10EAD00000DD09D608DC0DDC099643C6160FD70801
:10EAE0000E1A914327099643DE4E092731DF4E0F58
:10EAF000DE4A092611964C260D7C004CDE52DF467C
:10EB0000DE54DF4820D79C5026D30E7F0008DC540B
:10EB10009348DD54DC52D2479246DD5238397F00AB
:10EB200008CC0000DD52DD543839BDE52F7F005A96
:10EB3000DC522A06CC00137EEF0F3C2715740052DE
:10EB40007600537600547600557C005ADC5226ED50
:10EB50002011DC5427DE2B0B7800557900547A0005
:10EB60005A20EF7F00467F0047DC54C3B172DD4876
:10EB70007C0047CCB172DD52CC17ADDD54BDF086C0
:10EB8000DC54DD567F0058DC4FDD52965197547FA0
:10EB90000055BDF086DC54D357DD57965689009753
:10EBA00056965680809756DC5805DD58DC565949F4
:10EBB000DD56730056DC574353C30001DD579656AC
:10EBC00089009756CE0000DC56DD54DD482A03CE7E
:10EBD000FFFFDF52DF46BDF164DC4EDD5EDD54CC6D
:10EBE000994BDD48CC0000DD46DD52BDF164DC4EC2
:10EBF000C3F622DD54DC5EDD48CC0000DD52DD468C
:10EC0000BDF164DC4EC3E2A8DD60CC0002DD5EDC59
:10EC100057DD544FD6562A0286FFDD52DC54363774
:10EC200005DD58DC5236375949DD56CC0000DD464B
:10EC3000974896609749BDF164DC4FD358DD58DCA6
:10EC400056C9008900DD564FD64E2A0286FFD3569C
:10EC5000DD56D661D7493332DD523332DD54BDF152
:10EC600064DC4ED358DD58DC56C9008900DD564FB0
:10EC70005F7D004E2A03CCFFFFD356DD56DC578361
:10EC8000875DDD539656820097524F965A9B529756
:10EC900052DC53DD5436374FD6522A0286FF3637C0
:10ECA000DD5286B19749CC0000DD469748BDF1643E
:10ECB000DC4EDD56DC50DD58C672D7493332DD52AA
:10ECC0003332DD54BDF164DC4ED357DD548600D6BB
:10ECD000562A0286FFC90089007D004E2A03C3FF21
:10ECE000FFDD523839BDE52FDC522B0B83000A259E
:10ECF00006CC00147EEF0FDC52DD56DC54DD58DC10
:10ED000053DD5496529753CC0001DD46CC62E4DDCE
:10ED100048BDF164D64E2A0CC1F02408CC0000DDB9
:10ED200052DD54394F5CD75A2A0286FFDD5416DD76
:10ED300052CCB172DD487F00467F0047BDF164DCF4
:10ED4000509358DD54DC4ED2579256DD52DC524778
:10ED500056DD5EDC544656DD608607975B3CCCFF93
:10ED6000FFDD52CCFFF3DD54CEEDCFBDED9B7A003D
:10ED70005B26F8965A2B13270F78005579005479A3
:10ED800000537900524A26F1383977005276005301
:10ED90007600547600554C26F13839DC5EDD46DCD1
:10EDA00060DD48BDF164965048DC4E5949DD54CCD5
:10EDB00000007D004E2A03CCFFFFDD52EC02D3544D
:10EDC000DD54EC00D9539952DD5208080808390087
:10EDD00000005BFFFFFDDE00000AABFFFFD5550022
:10EDE000008000FFFF000000010000160908A600D7
:10EDF000812027F908112701093908A60081202759
:10EE0000F939BDF2A17EF2C60908A600812027F9D2
:10EE1000813F262608A600812027F981282705CCD6
:10EE200000400C39BDE52FDC522627DC544D26224C
:10EE3000C106241E0505C373B0398040240139265C
:10EE40002008BDE52FDC522609DC5418BC72881856
:10EE50002506CC00027EEF0F05054353C372190C43
:10EE600039811B25020D39084848164FC3721839DD
:10EE7000BDEF8E7F0044BDEDFB7F0046812626035B
:10EE80007EEF308130240139813A250139840F7DAC
:10EE90000044260A7C0044975508A60020E57C0023
:10EEA00044D644C10524149747DC5405DD540505B8
:10EEB000D354D346DD5408A60020C89747DC540538
:10EEC000DD54DD50DC5259492B42DD52DD4E7800D5
:10EED0005179005079004F79004E2B3078005179EC
:10EEE000005079004F79004E2B22DC54D350DD5472
:10EEF000DC52D94F994E2B14DD52DC54D346DD54ED
:10EF0000DC52C90089002B04DD5220AACC00033C4E
:10EF1000CEEF167EF2CC484F573F20204552524F3D
:10EF200052202300574841543F0D534F5252590D20
:10EF300008A600814827090939964426020909399B
:10EF400008A600803025F2810A250A8007810A255B
:10EF5000E8811024E47C0044D644C10924AEC604F0
:10EF60007800557900547900537900525A26F19B64
:10EF70005597557EEF40730052730053DC54435352
:10EF8000C30001DD54DC52C9008900DD52397F0025
:10EF9000527F00537F00547F0055393CFE738C3CF8
:10EFA000CEEFC3FF738CBDEFD938FF738C38393C7B
:10EFB000FE738C3CCEEFC3FF738CBDF04438FF73FF
:10EFC0008C38390001004441544146494C45204F9A
:10EFD00056455252414E4745003CBDEFDF38393669
:10EFE0007D00642609DC650525048102250B329D20
:10EFF000943838CC00047EEF0F331807360F1837DB
:10F00000D617C4F81B4C330F308C010125059F68BF
:10F010008E00FF971737DC66847FC340001832A745
:10F0200000D617C4F8D717308C010026029E681648
:10F03000320637DC66C30001DD66DC64C900890086
:10F04000DD6432393CBDF04A38397D00642609DC84
:10F05000650525048102250A9D973838CC00057E78
:10F06000EF0F16073617D617C4F81B4C0F308C015C
:10F070000125059F688E00FF9717DC66847FC340DB
:10F080000018A600209BDE46264BDE4826083838AE
:10F09000CC00067EEF0FDE52263BDC54CE00007C17
:10F0A000005278004979004824F5760048760049F6
:10F0B00093482404D3482001087A0052270B1805EE
:10F0C0001874004876004920E7DF54CE0000DF5274
:10F0D000DF4EDD50397F004ADE52DF4EDE54DF5016
:10F0E000CE0000DF52DF547C004A780049790048A6
:10F0F00079004779004624EF76004676004776008F
:10F1000048760049DC509348DD50DC4ED2479246A9
:10F11000DD4E2410DC50D348DD50DC4ED9479946F3
:10F12000DD4E20127C0055240D7C005424087C0008
:10F130005324037C00527A004A271A78005579003C
:10F14000547900537900527400467600477600489F
:10F1500076004920AF393CCE004686106F00084A41
:10F1600024FA38397F00447D00522A067C0044BDD1
:10F17000EF767D00462A1A7A0044730046730047F2
:10F18000DC484353C30001DD48DC46C9008900DD8B
:10F1900046BDF1BA964E2A06CC00077EEF0F964484
:10F1A000271773004E73004FDC504353C30001DD3B
:10F1B00050DC4EC9008900DD4E397F004E7F004F84
:10F1C0009649D6553DDD50D655272F9648270B3DFD
:10F1D000D34FDD4F964E8900974ED6559647270A56
:10F1E0003DD34EDD4E24037EF278D6559646270A4F
:10F1F0003D4D26F3DB4E25EFD74ED65427389649A2
:10F20000270B3DD34FDD4F964E8900974ED654962F
:10F210004827083D4DD34E25CEDD4EF6C42FC145BF
:10F220002614D6549647270A3D4D26BBDB4E25B7FC
:10F23000D74E964626B1D6532723964927093DD364
:10F240004EDD4E2533974ED6539648270A3D4D2620
:10F2500027DB4E2523D74E96479A46261BD65227A4
:10F26000169649270A3D4D260FDB4E250BD74E96A5
:10F27000489A479A46260139CC00077EEF0FBDEE2B
:10F280000825433736863DBDEDEB263ABDE2E3DF88
:10F2900046380FDC52ED00DC54ED020EDF52DE4644
:10F2A00039863ABDEDEB260532327ECB05860DBDA3
:10F2B000EDEB26063232087ECACF39BDEDFB810D5B
:10F2C00027F8813A27F43C4F5FCEEF240EDD547FC0
:10F2D00000527F0053CCF8EBDDAC7F00B57D0081A0
:10F2E00027273CFE738C8CFFFF38271D96B68118AC
:10F2F0002606BDF8EB7F00B68EBFFFCC0000FD7385
:10F300008EFD7394DE82BDCADD7F00B37F00B496AC
:10F31000B6270CBDF8EB96B6811826037F00B64FD2
:10F32000BDF464860AB7B59ADC5427097F0045BD51
:10F33000F49FBDF5E3FE738C8CFFFF26037ECDE5C5
:10F34000EC0026037EC716BDF539183809DF4618CC
:10F35000A600810D270FBDF5E59C462605863FBD1D
:10F36000F5E50820EBBDF5E57EC7163CCEEF2A4F4C
:10F370005F7EF2CCC60DD74636DF5218C300F0DDF3
:10F3800054DE52BDF8AE817F27418108273D810AB6
:10F3900027F1810027ED810326113337C13A260B6F
:10F3A00033383838FF738C387EF606A7000891464C
:10F3B000261233C13A270CBDF8EB810D2605860ACB
:10F3C000BDF8EB39BDF8EB9C5426B89C5227B40924
:10F3D0008608BDF8EB8620BDF8EB8608BDF8EB206B
:10F3E000A2DE548C80002508CC00087EEF0F32325C
:10F3F000CE73D2BC73A225040D86FF39EC00847F46
:10F400009354250139E602DF564FD3561820E420E5
:10F410000108A6002AFB20DB3CDE52270738CC007F
:10F42000087EEF0FDE548C800024F2FE738CEC001B
:10F43000847F26035D27B7189C543825D2FE738C31
:10F44000200C09E6000886FF50DF56D35618DC541E
:10F450008A80A1002605E1012601398C73D226E2BB
:10F460000D86FF3916A60008112601393637BDF57D
:10F47000E53332810D26EE398622BDEDEB260ABD3D
:10F48000F464810D2601094F398627BDEDEB27EF86
:10F49000817F260A81082606860D9DAB20E9393C2E
:10F4A000964536848097449645847F9745861436E2
:10F4B0007A0045F6B59AC10A260E7D00522A09BD8A
:10F4C000EF767C00447A0045F6B59A4F18DF487F06
:10F4D00000477F0046BDF086DE522604DE54270832
:10F4E000D651377A004520E0D651377B8044271526
:10F4F000964484012704862D9DAB7A00452B1B86FC
:10F50000309DAB20F57A00452B0686209DAB20F57B
:10F51000964484012704862D9DAB328114270C81EB
:10F520000A25028B078B309DAB20EF329745383987
:10F53000BDF5394FBDF4640839EC00847FDD547F9C
:10F5400000527F005308080886049745BDF49F8643
:10F5500020BDF5E539FE73A4BC73A8260139A600C9
:10F56000083CFE73A6A70008FF73A63820EAFE73C6
:10F57000AABC73AE26013909A6003CFE73AC09A7EC
:10F5800000FF73AC3820EA3233DF5E38FF73942714
:10F590001838FF739A38FF739C38FF739638FF73DF
:10F5A0009838FF739E38FF73A03736DE5E393233EA
:10F5B000DF5E308CB5FF2405DE5E7EF36BFE739458
:10F5C000271BFE73A03CFE739E3CFE73983CFE73AB
:10F5D000963CFE739C3CFE739A3CFE73943C37361B
:10F5E000DE5E39860D369DAB3236810D2604860AE5
:10F5F0009DAB32397D00932601397D009E27FA7F2D
:10F600000093BDF84C0E7D008C271A8EBFFDCC00F8
:10F6100000FD738EFD7394CC0064DD54CC0000DDDE
:10F62000523C7ECB14FE738C2727CEF654BDF5E3F7
:10F630004FBDF464FE738CEC00847FDD547F005278
:10F640007F00537F0045860AB7B59ABDF49FBDF58C
:10F65000E37EC716425245414B204154204C494E4F
:10F660004520000F36BDF76032843F8A8016BDF614
:10F6700095C6EBD71671DF17BDF767D756BDF7678D
:10F68000D757BDF757C6FBD7160E39BDF69571DFB4
:10F690001771BF173971DF1771BF1771EF177240FC
:10F6A0001772201771DF177210177220178608BDA6
:10F6B000F78A390F36BDF76032843F36C630BDF663
:10F6C0008B32368AC016BDF695BDF6F00E01010FDD
:10F6D00032843F8A4016BDF695D656BDF788D65778
:10F6E000BDF788BDF6F0C600BDF68BBDF7570E39E5
:10F6F00071EF1771DF1771BF17CE02627220170109
:10F7000001010171DF170926F3724017722017718A
:10F71000DF1771BF1739B6C4308154270AC11C27BF
:10F7200006C1182702D643BDF760BDF731BDF757B4
:10F73000390F9F688E00FF71BF17722017585858F5
:10F740008605BDF78AC6EBD71671DF17BDF767864A
:10F75000FB97169E680E399617840F8A8097173983
:10F76000710F1772401739C60272201771DF177BAD
:10F77000101727015C7220175824F171DF177B10D6
:10F780001727015C7220173986085871DF1772102D
:10F7900017250371EF177220174A26EE3996113696
:10F7A00084C0274C844027049612323BDE719612A7
:10F7B000A7007B0176271281132605728076203000
:10F7C00081112605717F762027810326037C009313
:10F7D000098C728B2603CE738BDF717D007526102A
:10F7E000189373C14026098613BDF8EB86FF977501
:10F7F000328424812427013B7B017627237B80767A
:10F80000271EDEAFBDF5F471FB110E010196431A00
:10F81000914327F90F0927057B807626E7717F76CC
:10F82000FEB596A600098CB4932603CEB593FFB51A
:10F83000967D007726029713FEB596BCB5942604F4
:10F8400071FB113B7204113B86FF97753CCE738BA5
:10F85000DF71DF7371FB11CEB593FFB594FFB596E1
:10F86000967527088611BDF8EB7F007538717F7695
:10F870007F0093399674907239B6B597B0B59539C3
:10F88000DE643CDE663CDEB3EC00DD64EC02DD668B
:10F890003CBDF04438D664E700D665E701D666E79C
:10F8A00002D667E70338DF6638DF643338393C3720
:10F8B00036DCB33226CADE739C7126031A20F7A603
:10F8C0000036098C728B2603CE738BDF73967527F7
:10F8D0000F189371C14026088611BDF8EB7F0075A3
:10F8E000323338810326037A0093393C3736FCB52E
:10F8F00096B3B594C1FF27F6FEB59432A700098CE4
:10F90000B4932603CEB593FFB594720411333839FE
:10F9100086209DAB86209DAB393B3B717F1BDE6C07
:10F9200008DF6CDC42C30001DD42DC40C900890015
:10F93000DD4096AE890097AE3B7B201127FB9713E5
:10F94000399614848027037EFA0D860397908E00E3
:10F95000FDBDF9641A1A1ACE0000DF42DF407F00B5
:10F96000AE7EC6938612971BB6C42E8B0C971C7F57
:10F9700000017F00207F008B7F008A860A97118616
:10F9800005971086E097148680971786FB97168652
:10F99000039790867EB7010FCCF91BFD01107240D2
:10F9A0001B0E86FF97777F0017722017720817C605
:10F9B000B1BDF788C6B2BDF788B6C43197177208D3
:10F9C00017C6A0BDF7888607365FBDF788324A267E
:10F9D000F77F008D7F008E7F008F86809717390F0D
:10F9E00097549610369603369615369614369F52CF
:10F9F00096148A8097147F0017722017720817C612
:10FA0000B2BDF788D654BDF788868097179E5232CC
:10FA100097148612971BB6C42E8B0C971C32971521
:10FA2000329703968B9720968A9701CE0000DF428B
:10FA3000DF407F00AE860A971132971086809717B5
:10FA400086FB971672401B0EBDF848861A9711392F
:10FA50002A202050433D2420413D2420423D2420A3
:10FA6000463D2420583D242040583D242053503DFD
:10FA700024204024DEAC3CCEF8EBDFAC0E860DBD7E
:10FA8000F8EB860ABDF8EBCEFA50BDFB0C3C30EC2F
:10FA9000091809BDFB1438BDFB0C3C30A606BDFBA4
:10FAA0001938BDFB0C3C30A605BDFB1938BDFB0C5D
:10FAB0003C30A604BDFB1938BDFB0C3C30EC0718EC
:10FAC000BDFB1438BDFB0C3C30EC0718EC0018BD36
:10FAD000FB1438BDFB0C3C3018C3000A18BDFB14E6
:10FAE00038BDFB0CFE7282BDFB14863DBDF8EBFEFB
:10FAF0007282860836A60008BDFB198620BDF8EB89
:10FB0000324A26F038DFAC3BBDF8EB08A600812472
:10FB100026F608393C328D013236444444448D0186
:0EFB200032840F8B30813A25028B077EF8EB82
:10FFCA007EF7317EF7607EF7577EEF9B7EEFAF7E3E
:10FFDA00F8747EF8AE7EF8EB7EF84C7EF71600C118
:10FFEA000100010FF919F79D010301060109010C2E
:06FFFA00FA74F91AF94146
:00000001FF
